:100000007003012055180000531800005318000019
:10001000531800005318000053180000000000009F
:100020000000000000000000000000005318000065
:10003000531800000000000053180000531800007F
:100040005318000053180000531800005318000004
:1000500053180000531800005318000053180000F4
:10006000531800005318000053180000B519000081
:1000700053180000531800005318000053180000D4
:1000800053180000531800005318000053180000C4
:1000900053180000531800005318000053180000B4
:1000A00053180000531800005318000053180000A4
:1000B0005318000053180000531800005318000094
:1000C0005318000053180000531800005318000084
:1000D0005318000053180000531800005318000074
:1000E000531800005318000000000000000000003A
:1000F00000000000191800005318000053180000F9
:100100005318000053180000531800005318000043
:100110005318000053180000531800005318000033
:100120005318000053180000531800005318000023
:100130005318000053180000531800005318000013
:100140005318000053180000531800005318000003
:1001500053180000531800005318000053180000F3
:1001600053180000531800005318000053180000E3
:1001700053180000531800005318000053180000D3
:1001800053180000531800005318000053180000C3
:1001900053180000531800005318000053180000B3
:1001A00053180000531800005318000053180000A3
:1001B0005318000053180000531800005318000093
:1001C0005318000053180000531800005318000083
:1001D0005318000053180000531800005318000073
:1001E0005318000053180000531800005318000063
:1001F0005318000053180000531800005318000053
:100200005318000053180000531800005318000042
:100210005318000053180000531800005318000032
:100220005318000053180000531800005318000022
:100230005318000053180000531800005318000012
:100240005318000053180000531800005318000002
:1002500053180000531800005318000053180000F2
:100260005318000010B5054C237833B9044B13B173
:100270000448AFF300800123237010BD70000020FC
:1002800000000000C031000008B5034B1BB103495A
:100290000348AFF3008008BD000000007400002098
:1002A000C031000070B50D461646044610B1081E58
:1002B00018BF01200549064B34229847236832466F
:1002C00029462046BDE87040184700BFE42A0000D8
:1002D0000516000070B50D461646044610B1081EFE
:1002E00018BF01200549064B3D22984763683246F6
:1002F00029462046BDE87040184700BFE42A0000A8
:10030000051600004FF0E0236FF07F425A6105228E
:100310001A61704738B5044600380C4B0D4618BFBB
:1003200001200B494FF4E07298472368AB4208D094
:100330004BB9084B25602046984740F2B273A36141
:1003400038BD0020FCE76FF01100F9E7051600004A
:10035000F82A00003919000037B5134D0020A847CE
:1003600004460028FAD1114DA84782070BD0104B44
:1003700001222146204698470E4B0F4801219847FD
:100380000E4B204698470020A847430709D516235F
:1003900000220193084B0093094C0123114610469B
:1003A000A04703B030BD00BF21070000090D0000C9
:1003B0002D0D0000B10D00008C000020010E00008A
:1003C0005D0E0000024A0348034B111D184700BF91
:1003D000000000201C03002009070000044A1168E7
:1003E000034609B90349116010680344136070475C
:1003F0008C02002070030120891A70B5CC1D48BF03
:1004000001F10E0400EBE40002F0070210F8011CF9
:10041000D418082C41FA02F118DD10F8025CC2F180
:100420000806B540102C41EA05010FDD10F8030C59
:10043000C2F11005182CC8BFC2F1180200FA05F568
:1004400041EA0501C4BF00FA02F211434FF0FF3048
:10045000984021EA000070BD37B50E4B054601A853
:1004600098470D4A6B09D90102EBC31351581A6A18
:100470001C690A4B54400C4001A8544005F01F056C
:100480009847012000FA05F5254208BF002003B077
:1004900030BD00BF9920000000800041A72000006F
:1004A00013B50748074C0268917F537B003918BF8A
:1004B00001210091017912688068A04702B010BD47
:1004C00090020020F913000038B5002843D1234CD6
:1004D000E368002B38D0B3F90000421C34D0204B25
:1004E000C0B29847E3685B88984203D00423A376A0
:1004F000022038BDA07E042801D10123F7E701289E
:100500001FD10223A376174B2361012363770023B6
:1005100084F82E302379E3B1208EB0FA80F04009C0
:10052000114A1249124D40F22C53A847002323715F
:10053000104B2360104B9847A07E831E58425841B1
:10054000D7E70328E6D1D4E7A37E033B012BE1D80C
:10055000D7E70120E4E70420CBE700BF90020020AA
:1005600059040000801A0600122B0000252B000001
:1005700069210000A0020020A10400002DE9F04143
:100580000B4D0C4E0C4FDFF834803368B0681A897D
:1005900041F20D111204B847044628B1B068C047B3
:1005A000C30502D4013DF0D100242046BDE8F0810E
:1005B000410D03009002002049120000B913000011
:1005C00073B50E4C0E492368A0681A890D4E01259B
:1005D0001023CDE900559A40B04760B12168A0686A
:1005E000094B2A460E31984728B1A068074B02B044
:1005F000BDE870401847002002B070BD9002002096
:1006000009110800611000005D12000009130000CC
:10061000034B197911B99868024B1847704700BF0E
:1006200090020020111400002DE9F7430546DFF881
:1006300070900A9F0E4690461C46134A134940F29A
:1006400095430120C847104A104940F296430120C3
:10065000C847A30643EA482444EA0672C7F30801E0
:100660000B480C4C0A4301230B49CDE90033002D04
:1006700008BF01460948BBB242EAC5728068A0477C
:1006800003B0BDE8F08300BF122B0000252B000053
:100690003513010061100000359301009002002025
:1006A000692100002DE9F0411D4606461446281E2A
:1006B00018BF01200E4ADFF84C800F4640F2764307
:1006C0000C496402C04744EA077242EAC6702A78BD
:1006D000094E0A4B024341F23431B0689847044650
:1006E00018B1B068064B984728702046BDE8F081E5
:1006F000122B0000252B0000900200204912000060
:10070000B91300006921000010B5044B04249C7645
:10071000FF241C71C3E902015A6310BD900200203E
:100720002DE9F04F844B89B098470128804605D0C9
:10073000824B9847404609B0BDE8F08F804C814F0E
:1007400023680025D8721D731D817F48B847A068B3
:100750007E4B98472A46A0687D4D4FF48851A847A4
:1007600038B3A0684FF4D57245F20851A84730BBA2
:100770000026A068002244F20551A847002800F096
:10078000A680A068DFF8CC91C84710F0E04F00F0D9
:100790009E8041F2893A00F4FC1244F20551A068AF
:1007A000A84730B1A068C847002814DBBAF1010A95
:1007B000F1D123684FF0030883F80A80B8E7A068F6
:1007C000644B9847411CD3D0C0F30B00B0F5D57FE4
:1007D000EFD14646CDE7020123682FD50522DA7214
:1007E0004FEA867A5B4E41F6EF39A068002241F26B
:1007F0003711A84700287FD157495848B84758486B
:10080000B8472368A0680222DA724FF488510022A8
:10081000A8470028CDD0DFF83C9141F6EE36A0681D
:10082000002241F20111A847002840F02A81C6F5B4
:10083000DF524C494C480E32B847BAE70422DA720C
:10084000DFF834A10DF114090926D34600214B46E7
:10085000324608460136D0470D2E09F10109F5D17F
:100860009DF815309DF8146006EB03269DF81630B0
:1008700006EB03469DF8173006EB036606F580731A
:1008800003934FF0000900210DF1180A0AEB090348
:1008900006EB0902084609F10109D847B9F1030F2F
:1008A000F1D19DF81830FF2B83D0222B04D19DF875
:1008B0001A30002B00F0FA819DF81930002B3FF41C
:1008C00078AF02331E44039B9E42DAD971E7236856
:1008D000DB7ADB0784D42368DB7A5A07B0D4236839
:1008E000DB7A03F00903012B00F002822368DB7A34
:1008F000DB0700F188818BE1A068524641F22911A3
:10090000A84710B91449194878E7A068B04710F013
:10091000010208D0B9F101097FF467AF02460E4920
:100920001348B8476BE7A06840F23A51A84728BB84
:100930000949104862E700BFC90400001106000021
:1009400090020020D5200000292B0000C5130000D4
:1009500049120000B91300000C2C0000412B0000CC
:10096000A22B00001B2C0000B62B0000522B000015
:10097000642B0000912B0000A5060000A068B04782
:10098000400004D52268D37A43F00803D372A068EC
:10099000002241F23B11A84700283FF40AAF236828
:1009A000DB7AD90797D5B24B984700283FF401AFBF
:1009B000D4F800A0AF4E0AF10E0B0823602280216C
:1009C0005846B047AC4BC0F3C30200F0070003EB3E
:1009D000800003EB82028021D36F026E53434FF4F9
:1009E0007A725343CAF800307E2202235846B04739
:1009F000B146002800F01E8116233022802158467F
:100A0000B04701304002BAF80820CAF804001204C6
:100A1000A06841F23711A84700283FF4CAAE01266A
:100A2000CDE900669549A068DFF86CA20823002292
:100A3000D04700283FF4BDAEA068914B324606A9CE
:100A4000984700283FF4B5AEA0688E4B9847002821
:100A50003FF4AFAE04233822402106A8C847B04275
:100A6000D4F800A000F0FD80022840F0FE8033465C
:100A70002F22402106A8C84701280CBF302320237D
:100A8000F0E0A068C84710F0010206D0013EBFF4B4
:100A9000C6AE7D497D48B8478BE6A06840F23A5122
:100AA000A84710B978497A48F5E7A068C84700F028
:100AB000C040B0F1804F08BF2268A06802BFD37A5F
:100AC00043F00803D37241F23B110022A8470028EB
:100AD0003FF46FAE664B984700283FF46AAED4F8F7
:100AE0000090644E09F10E0B04237A2280215846AF
:100AF000B0470138B246032803D8DFE800F09193ED
:100B00009597122389F80C306022082380215846DB
:100B1000D047594BC0F3C30200F0070003EB80003D
:100B200003EB82028021136A026E53434FF47A7200
:100B30005343C9F800303E220C235846D04740F6B4
:100B4000FF739842064612D003232F228021584675
:100B5000D047731C023003FA00F650220423802190
:100B60005846D04706FA00F0800AC9F8040099F800
:100B70000C303F2B3ED901230022CDE900324549FC
:100B8000A068454E4FF40073B04700283FF411AE03
:100B9000DFF814B13226D946A06805A9D847002845
:100BA0003FF407AE013EB6B2002EF5D120680C230B
:100BB0003E2280210E30D04740F6FF73984237D155
:100BC0000426A06806A9C84700283FF4F2AD013EFC
:100BD000B6B2002EF5D1069B22685B08536036261C
:100BE000A06806A9C84700283FF4E3AD0136B6B2B5
:100BF000802EF5D1A0684FF4007241F21011A84781
:100C000000283FF4D6AD254B984700283FF4D1ADDE
:100C1000234B98472348B847236800229A7287E5F8
:100C200014236FE722236DE730236BE7402369E746
:100C30003226D5E70C233E2280215846B0470323B5
:100C400006462F2280215846C8470136023086408A
:100C50000423502280215846C84706FA00F0800A33
:100C6000D1E61A238AF80C3035E61023FAE700BFE4
:100C7000C1050000F90300000C2C0000331108002E
:100C80005D120000091300001B2C0000DA2B00008D
:100C9000912B000008110800611000007D05000084
:100CA000A1040000F52B00000D13000006F1060959
:100CB00000215346324608460136D8474E450AF1D0
:100CC000010AF5D19DF81D300E492268322B28BF4C
:100CD000322303F00700DB0801EB800001EB830106
:100CE000036EC96F4B434FF47A714B431360F6E5C3
:100CF000A0684FF4007241F21011A84700287FF459
:100D0000F5AD56E50C2C000008B5054B984728B901
:100D1000044B9847044B1B68D87A08BD0020FCE7B9
:100D2000C90400001106000090020020F7B5174B1F
:100D30000F4614469847054628B9154B984728B9D9
:100D4000144B98470525284603B0F0BD124B134EAF
:100D50001349B068012C98BF19463368DB7A1B072A
:100D600058BF7F020123CDE900433A464FF4007398
:100D70000C4FB8470028E3D00B4BB06898470B4B9B
:100D80000340002BDCD134863487DCE7C904000043
:100D90007D050000110600001111080090020020DE
:100DA0001211100061100000B9130000000058E497
:100DB000F8B50E4D0E4A0F4F0646288E0C46A0423F
:100DC00034BF002001200C494FF4D963B847A8680C
:100DD0000A4B22463146984728B1288E011B89B21A
:100DE00000202986F8BD01460520FAE79002002080
:100DF000122B000069210000252B00005D1200006D
:100E000038B5124D124B0446A8689847E0B144B17A
:100E100000232B862B8F012B08D10E4B98470020E7
:100E200038BD2B8E002BF5D02046F9E70022A868AC
:100E3000094C43F20C11A04702460028EDD1A868E6
:100E400043F20C11A047E8E70520E9E790020020F3
:100E500009130000110600004912000070B586B0A9
:100E6000CDE90421BDF82C5003936C1EB4F5007F2E
:100E70001FD2114CA047044648B90095DDE9033262
:100E80000E4D0599A8470E4D20B9A84705242046C8
:100E900006B070BD0B4E0A99B0680B4B0122984703
:100EA0000028F2D0B068094B98470028EDD0A84739
:100EB000EDE70624EBE700BFC904000029060000A7
:100EC00011060000900200205D12000009130000CE
:100ED00073B5FF238DF802308DF8033000230193A2
:100EE00001A9174B174D184E184C984701220DF1C8
:100EF00003010198A84701220DF102010198B047B2
:100F000001220DF103010198A847019801220DF17A
:100F10000201B04701220DF103010198A847019891
:100F200001220DF10201B047013C06D09DF80230CC
:100F3000FF2BEFD1012002B070BD2046FBE700BFC0
:100F400021150000A5020000D5020000410D03009C
:100F50001FB50023039303A9094B9847FF238DF87E
:100F600007300DF107010398064B012298470398BB
:100F7000054B022202A9984705B05DF804FB00BFAB
:100F800021150000A5020000D50200002DE9F34163
:100F9000264B274D274EDFF8C480002401A9019479
:100FA0009847254A25491068FF238DF80330938818
:100FB000B0FBF3F203FB1200B0FA80F0204AB32337
:100FC0004009A8478DF802401E4C013C05D11E493E
:100FD0001E481F4B984720461FE001220DF10301D8
:100FE0000198B047019801220DF10201C0479DF818
:100FF000020010F0F00715D1003818BF01200F498A
:101000000F4AC923A8479DF802000F49104B10F062
:10101000070405D00F489847384602B0BDE8F08174
:101020000D48D7E7FE28D0D10120F6E721150000B2
:1010300069210000A5020000CC020020252B000041
:10104000C82C000021A107001F2F0000DF2C00008A
:10105000D5200000F92C0000142D0000D50200005E
:101060002DE9F04F89B00E460024029305A9664B86
:101070000594154682469847FF23644A644F8DF8CD
:1010800011308DF813306349F723C6F3002006F0C2
:101090003F09B84749F040038DF818302B0E8DF802
:1010A00019302B0C8DF81A3006AF2B0A8DF81B3037
:1010B0008DF81C50234606223C46013A12F0FF02EE
:1010C0002FD15B0043F00103DFF8748105988DF8A0
:1010D0001D3001220DF11101C0472146062205985D
:1010E0004D4FC047FF2305988DF8123001220DF1B6
:1010F0001201B8470724012205980DF11201B847E3
:101100009DF912309DF81220002B1EDA013C14F0DC
:10111000FF04F0D1414942482B464A46414DA84779
:1011200023E017F8010B08215B00DBB283EA000C17
:101130001CF0800F01F1FF3118BF83F0090340005C
:1011400011F0FF01C0B2EFD1B7E7DFF8F8B012F04D
:101150000803CBF8082003930BD0304932480092A3
:101160002B464A462F4CA0470024204609B0BDE834
:10117000F08F12F0040405D0009228492B482B462A
:101180004A46EFE712F0FE0F07D000922B462349A4
:10119000244D27484A46A847E7E7B10409D5254A20
:1011A00050469047044620B91C4923482B464A46DE
:1011B000B4E7B2050BD50022CBF808200DF11301DE
:1011C00001220598C0471D4905980122B8477305BB
:1011D0000DD501220DF113010598C04704221749CE
:1011E0000598B847DBF8082012BACBF80820BDF8FC
:1011F0004820029BABF806200022ABF80430CBF865
:1012000000200124B1E700BF21150000C82C000018
:1012100069210000E12D0000D5020000782F0000B8
:10122000042E0000D52000002C2E0000632E0000AC
:101230009C2E0000D10E0000CB2E0000D402002016
:10124000A5020000CC02002013B50023CDE9003335
:10125000014CA04702B010BD611000002DE9F74F0E
:10126000204B214DDFF89490DFF894A088460026AB
:1012700001A90746144601969847FF238DF80330CD
:101280001CB9012003B0BDE8F08FB5F806C02B688B
:10129000A888B3FBF0F0844594BF002001204FF4F0
:1012A000B2734A465146DFF85CB0D8470F4B384618
:1012B0009847013CA4B20028E4D00DF10301019845
:1012C0000B4B01229847AA8801980A4B08EB0601AC
:1012D0009847AA882B6813442B603846064B16445F
:1012E0009847CDE721150000CC0200208D0F0000AB
:1012F000A5020000D5020000510F0000C82C00001C
:10130000252B000069210000012070477FB5214C8A
:1013100001910023039303A91F4B05469847E688D4
:10132000A0881E4A1E49FF238DF80B302368B3FBAB
:10133000F0F086424FF4E7731A4E94BF002001206C
:10134000B047A2882368B3FBF2F102FB1133B3B1BB
:10135000154B039801220DF10B01984704220DEB68
:101360000201124B039898472368A2880433236034
:10137000B3FBF2F102FB113343B1012004E00C4B4B
:10138000284698470028E3D104B070BD094B284691
:101390009847F2E7CC02002021150000C82C00007D
:1013A000252B000069210000A5020000D5020000E5
:1013B0008D0F0000510F0000014B9868704700BF6F
:1013C000CC02002037B50023019301A9084B094D39
:1013D0009847FF238DF803300A24019801220DF16C
:1013E0000301013CA84714F0FF04F6D103B030BD5F
:1013F00021150000A5020000044AD2F8903023F025
:101400008053C2F890300020704700BF0080004138
:10141000044AD2F8903043F08053C2F89030002054
:10142000704700BF0080004138B50D46044610B13A
:10143000081E18BF01200A490A4B4022984720463F
:10144000094B40F8045F29469847002807DB4FF412
:101450000043A382054B2361054BE360002038BDA8
:10146000E62F000005160000A51E0000E91400008C
:10147000B114000030B50C4685B0054610B1081E09
:1014800018BF0120B3220749074B984723680193EF
:1014900063680293A368039301A9044B281D98472E
:1014A00005B030BDE62F000005160000D91F000072
:1014B0007FB50446003818BF01200E46154607497F
:1014C000074BA32298470023CDE9016301A9054BEF
:1014D0000395A4F10C00984704B070BDE62F0000FE
:1014E00005160000751400007FB50446003818BFCB
:1014F00001200E4615460749074B872298470023CF
:10150000019301A9054B0296A4F10C00039598479D
:1015100004B070BDE62F0000051600007514000031
:1015200038B50D46044610B1081E18BF0120044905
:10153000044BBD220C3498472C60002038BD00BFFE
:10154000E62F00000516000070B50D46044610B1E8
:10155000081E18BF01200549054B3122984729462E
:101560002046044BBDE87040184700BF0230000021
:101570000516000049160000014B1860014B184782
:10158000D8020020050300000A4A13889BB210B558
:1015900043F4A0631380084B9847084B9847084BC7
:1015A0009847084B9847BDE81040074B40F6FF703E
:1015B000184700BF00400041111900000B16000041
:1015C0000D1800000D160000CD150000C20707D54C
:1015D000094B0A4A1A6243F6FD7259681142FCD15E
:1015E000030707D5044B064ADA6243F6FD725968D1
:1015F0001142FCD1704700BF001C004007010100F0
:101600000501010000B900BE704770470C4B0D4A40
:101610005A63DA6B12F0060FFBD14FF402629A6341
:10162000022283F83020064AD36B9807FCD4044B7F
:101630001A6CD10702D41A6C9207F9D5704700BF13
:10164000001000404D0E010038B50C46054610B1A3
:10165000081E18BF0120124B1249D822984794F84F
:101660002F302C6043F0010384F82F3094F82F00C2
:1016700010F00100FAD10E2384F82E300F2384F8E5
:101680002930A38E9BB26FEA53236FEA4323A386CC
:10169000E38E9BB26FEA93236FEA8323E38638BD20
:1016A000051600001C3000002DE9F8430E461546D3
:1016B000044618B129B3101E18BF01201249134B5C
:1016C000134FF12298470834B9462046B8470028FE
:1016D000FBD0DFF844800027F15D2046C04720465C
:1016E000C8470028FBD00137BD42F5D8002D094E70
:1016F00008BF01252046B0470028FBD02846BDE89A
:10170000F8830846DAE700BF333000000516000012
:10171000871E0000911E0000791E00002DE9F8438D
:101720000E461546044618B1E9B1101E18BF012037
:101730000E490F4BDFF83C90DFF83C804FF4867287
:101740009847002708342046C8470028FBD0204689
:10175000C047F0550137BD42F5D8002D14BF2846CB
:101760000120BDE8F8830846E2E700BF33300000FF
:10177000051600009B1E00007F1E000038B50D46B8
:10178000044610B1081E18BF01200749074B342238
:101790009847074B294604F10800984718B9054BAC
:1017A0006360054B236038BD333000000516000030
:1017B000391E00001D170000A916000010B50446D0
:1017C000003818BF01200549054B5322984704F102
:1017D0000800044B9847002010BD00BF33300000C4
:1017E00005160000651E000038B50D46044610B110
:1017F000081E18BF01200349034B692298472C603B
:10180000002038BD3330000005160000014B0122D6
:101810005A717047000800400B4A937882B0DBB2DF
:101820000193019B990705D5084B1B6813B15068BC
:1018300002B01847019BDB0704D5044B5B680BB172
:10184000014AF4E702B0704700000241DC020020C8
:101850007047FEE718491948814210B50AD0184B65
:10186000DA1C121A22F00302C41EA34238BF00225F
:10187000144B9847144B1548DA1C121AC11E22F05B
:101880000302994288BF0022114B00219847114A58
:10189000114B22F07F029A60D3F8882042F4700244
:1018A000C3F88820BFF34F8FBFF36F8F0B4B984760
:1018B0000B4B9847FEE700BFC0310000000000203E
:1018C0006C000020CD2100006C030020700000207F
:1018D000E92100000000000000ED00E0852100008B
:1018E000E518000008B5054B9847054B9847054B90
:1018F00005489847054B9847FEE700BFB520000014
:1019000035210000D52000004F30000059030000B1
:10191000064B42F28E329A8200229A75DA75DA69A3
:1019200002F47C52DA6101221A74704700140040FC
:1019300003690B42FCD1704710B5044618B100682A
:10194000003818BF01201749174B2F229847174B13
:101950002068174A1C6048F20301904703889B07E0
:101960000AD52068038823F002031B041B0C0380A4
:101970009047206802219047206803889BB243F07B
:1019800001030380012190472068904720684FF4AD
:101990000143038048F20301904723680020186642
:1019A00010BD00BF5C30000005160000EC020020F6
:1019B000311900000D4B10B51C68226891895389BC
:1019C0009BB20B40DA0507D5636820469847236829
:1019D0004FF480729A8110BD5B04FCD5A368204649
:1019E000984723684FF48042F4E700BFEC020020E0
:1019F00000F01F0330B501259D4040090D4BC0018B
:101A00000229ACB24FEA154203440BD044F08044A3
:101A100044F4003442F040425D6042F400329C6283
:101A20009A6230BD44F080449D6042F040429C6226
:101A3000F6E700BF00800041420900F01F0303EBFE
:101A4000C21303F1824303F5004393F8402002F0F0
:101A5000FB0283F8402070474309DB0103F1824316
:101A600030B503F5004300F01F041D1903EB5403C8
:101A700095F8402002F0FE0242F0010285F8402075
:101A8000CAB293F8301010F0010F1BBF01F00F0124
:101A900041EA021101F0F001C9B208BF114383F815
:101AA000301030BD024A536943F4007353617047EC
:101AB0000008004010B5044B044905489847BDE8AC
:101AC0001040044B184700BFA51A00000024004036
:101AD000F00200201503000010B5054C054939201F
:101AE000A04723460449BDE810403820184700BFEE
:101AF000591A00000300390003003800064B402249
:101B0000C3F8DC204322C3F88C20044A936943F4D1
:101B100000739361704700BF001C00400008004044
:101B200010B5054B054906489847064B00229847D3
:101B3000BDE81040044B1847FD1A00000020014189
:101B4000100300207D170000D91A000070B5114E57
:101B5000114D124C4FF00063C6F8943002213B2027
:101B6000A8470F493B20A0474FF08063C6F8943048
:101B700002213A20A8470B493A20A04701213D20E5
:101B8000A847094B09493D2098472346BDE87040C6
:101B9000184700BF00800041F1190000591A0000E9
:101BA00003003B0003003A00391A000003003D0027
:101BB000064B4022C3F808214322C3F88C20044A74
:101BC000136A43F001031362704700BF001C00401A
:101BD0000008004010B5054B054898474FF0864176
:101BE000044B9847BDE81040034B1847B11B000059
:101BF0001C030020291400004D1B00002DE9F047B4
:101C0000214E224F224D234C4FF4006902212B20FC
:101C1000B8472B202049C6F89490A847A047022136
:101C20000820B8474FF48073736108204FF0081103
:101C3000A847A04702210920B8474FF400737361F9
:101C400009201649A8474FF48068A04702210A20BE
:101C5000B8470A201249C6F81480A847A0470221B5
:101C60000B20B8470B200F49C6F81490A847A0478F
:101C700002212A20B847C6F894802A20A8470A499A
:101C80002346BDE8F047184700800041F1190000E5
:101C9000391A0000591A000008002B00080009003A
:101CA00008000A0008000B0008002A00054A136912
:101CB00043F400431361044B4022C3F83421C3F8BA
:101CC0008C20704700080040001C004010B5054BF8
:101CD000054898474FF08A41044B9847BDE81040AB
:101CE000034B1847AD1C00003803002049150000C5
:101CF000FD1B00000148024B184700BF10E000E048
:101D00007915000010B5074B9847074B9847074BCC
:101D10009847074B9847074B9847BDE81040064B3C
:101D2000184700BF89150000B51A0000211B0000EC
:101D3000D51B0000CD1C0000F51C0000C3690B4240
:101D4000FCD17047C3690B42FCD170470268034B5A
:101D500022F0020202600321184700BF3D1D00006F
:101D60000268034B22F0020202600321184700BF01
:101D7000451D000070B50C4D06460FCD88B06C4671
:101D80000FC495E80F0084E80F006A46002352F85C
:101D9000041BB14202D1D8B208B070BD0133082B88
:101DA000F5D10020F8E700BF8C30000038B51B4BA0
:101DB00004469847022805D019491A4B40F2472299
:101DC00000209847E369184D13F0010F0ED103214D
:101DD0002046A84723689B0703D5144B9847022148
:101DE000A8470523236003212046A8472046012158
:101DF000A8470F4B23600321A8474FF4403363608B
:101E00001F21A8470B4BA3604FF61143A38100236A
:101E1000A373184684F8303038BD00BF751D00002C
:101E20007130000005160000451D0000611D000016
:101E3000040010400200700070B5054600380C46E2
:101E4000054B064918BF0120BB2298472C6020464D
:101E5000034BBDE8704018470516000071300000C4
:101E6000AD1D00000068036843F002030360032116
:101E7000004B1847451D00000368996270470368CE
:101E8000986AC0B270470368187E00F0010070477E
:101E90000368187EC0F3400070470368187EC0F3E3
:101EA000800070472DE9F843444B454D07460846EE
:101EB0000C469847042818BF0025002F5DD0201E2F
:101EC00018BF01203F4E404940F63F12B047B04690
:101ED000002D70D0E3693D4E13F0010F13D10321A3
:101EE0002046D5F80090B04723689B0709F01C09ED
:101EF00003D5374B98470221B04749F001032360CF
:101F000003212046B04701212046B0472B68DFF867
:101F1000C4903C6003F01C03082B30D12A490120F7
:101F200040F61D12C0472B6803EA09032360032112
:101F30002046B0476B6823F4083323F4107343F44E
:101F4000003343F4107363601721B047AB686362DA
:101F50006B7B84F83030E369002BFCD16B6813F0A5
:101F6000070F0CBF012302233B71AB7BEA7B43EAE3
:101F70000223FB800020BDE8F8833846A2E712491F
:101F8000012040F60912C0472B6803EA09032360C9
:101F900003212046B0476B6823F4383323F41073D1
:101FA00043F4003363601721B0472B7B23736B7BB3
:101FB00084F83030D2E76FF00C00DCE7751D0000CC
:101FC000C430000005160000713000003D1D000007
:101FD0004D1D0000FCFEFFFF2DE9F843046890F85A
:101FE00004802A4B0746201ED1E9006540F6A32253
:101FF00018BF0120894626499847E26912F0070276
:102000003ED1244B032120469847236899073AD5AF
:102010001146237ED8B25B070FD48A4218D8C30773
:1020200016D5FB8836B1B8F1010F33788CBF36F87E
:10203000023B01360132A3620AE0A36A3DB1B8F166
:10204000010F2B7085BF1B0A6B7001350235013102
:10205000000607D4D9F808309342DAD88B42D8D892
:10206000104606E04FF6FF736383802323766FF0FC
:102070001200237E9B07FCD003232376BDE8F88360
:102080006FF00300FAE76FF01300F7E705160000A2
:10209000713000003D1D0000EFF31083036072B645
:1020A000BFF35F8F7047BFF35F8F036883F31088C0
:1020B0007047000010B5044B9847044B9847BDE8A3
:1020C0001040034B184700BF051D0000C50300006A
:1020D000511800000FB430B5C3B0114C469D2846CE
:1020E000A047FF2818D80F4B4FF48072002102A898
:1020F000984747AA0C4B0192294602A8984702A884
:10210000A0470A4B82B202A91868094B984743B00E
:10211000BDE8304004B070474FF0FF30F7E700BF34
:10212000F9210000E92100003522000050030020C1
:10213000A502000010B5064C0649074B20469847FB
:10214000064B20469847064B06489847002010BD8E
:102150001003002050030020E9170000BD17000005
:10216000D5200000D530000010B50C46194620B926
:1021700023460248024CA047FEE710BDE8300000AD
:10218000D520000070B50D4D0D4C641BA410002629
:10219000A64209D10B4D0C4C01F002F8641BA410AF
:1021A0000026A64205D170BD55F8043B984701367C
:1021B000EEE755F8043B98470136F2E7AC310000F2
:1021C000AC310000AC310000B03100000A44914253
:1021D00000F1FF3300D1704710B511F8014B03F83F
:1021E000014F9142F9D110BD02440346934200D100
:1021F000704703F8011BF9E7034613F8012B002A87
:10220000FBD1181A0138704700B59BB000910491BA
:102210006FF000410591029105490391694600F074
:10222000CBF8009B00221A701BB05DF804FB00BFC6
:102230000802FFFF13460A46014602480068FFF7FE
:10224000E3BF00BF0800002070477047F8B5CD1C01
:1022500025F0030508350C2D38BF0C25002D06464A
:1022600001DBA94203D90C2333600020F8BD00F044
:10227000B1FB21490A6814469CB9204F3B6823B939
:102280002146304600F02CFB38602946304600F0ED
:1022900027FB431C23D10C233360304600F0A0FB06
:1022A000E3E723685B1B17D40B2B03D923601C4483
:1022B000256004E06368A2420CBF0B6053603046A7
:1022C00000F08EFB04F10B00231D20F00700C21A62
:1022D000CCD01B1AA350C9E722466468CCE7C41CC3
:1022E00024F00304A042E3D0211A304600F0F8FAAB
:1022F0000130DDD1CFE700BF540300205803002098
:102300002DE9F0478E689E4282460C4690461F4655
:1023100038D88A8912F4906F32D025680969A5EB04
:102320000109656905EB450505EBD57501334B449E
:102330006D109D4238BF1D46530531D52946FFF724
:1023400085FF064650B90C23CAF80030A38943F034
:102350004003A3814FF0FF30BDE8F08721694A4672
:10236000FFF734FFA38923F4906343F08003A38134
:10237000266165614E44A5EB09052660A5603E46D1
:10238000BE4200D93E4632462068414600F008FB76
:10239000A36822689B1B3244A36022600020DBE715
:1023A0002A4600F071FB06460028E1D1216950461B
:1023B00000F01CFBC7E700002DE9F04F98468B8921
:1023C0001B069DB007460D4614460ED50B6963B932
:1023D0004021FFF73BFF2860286120B90C233B60B8
:1023E0004FF0FF30D1E040236B610023099320239D
:1023F0008DF82930CDF80C803023DFF8A8818DF8D6
:102400002A304FF0010923469A4613F8012B0AB1EE
:10241000252AF9D1BAEB040B0BD05B46224629469C
:102420003846FFF76DFF013000F0AA80099A5A4440
:1024300009929AF80030002B00F0A28000234FF0A0
:10244000FF32CDE905230AF1010A049307938DF8C1
:1024500053301A935446052214F8011B514800F0DA
:102460004FFA049AD8B9D00644BF20238DF85330D0
:10247000110744BF2B238DF853309AF800302A2BD4
:1024800015D0079A544600204FF00A0C214611F847
:10249000013B303B092B4ED9B0B1079214E0A0EBC1
:1024A000080309FA03F313430493A246D2E7039BFC
:1024B000191D1B680391002BBBBF5B4242F0020257
:1024C00007930793B8BF049223782E2B0CD163781F
:1024D0002A2B35D1039B1A1D1B680392002BB8BF12
:1024E0004FF0FF3302340593DFF8C8A021780322B0
:1024F000504600F005FA40B14023A0EB0A0003FA71
:1025000000F0049B03430134049314F8011B264894
:102510008DF82810062200F0F3F9002838D0234B5C
:102520001BBB039B073323F0070308330393099B6B
:102530003344099367E70CFB02320C460120A5E700
:1025400000230134059319464FF00A0C204610F879
:10255000012B303A092A03D9002BC5D00591C3E7D6
:102560000CFB012104460123F0E703AB00932A464C
:102570000F4B04A93846AFF30080421C0646D6D163
:10258000AB895B063FF52CAF09981DB0BDE8F08F15
:1025900003AB00932A46064B04A9384600F07AF8AC
:1025A000EBE700BF6C310000763100000000000056
:1025B00001230000723100002DE9F04716469946CC
:1025C0008A680B69DDF820809342B8BF13463360F8
:1025D00091F8432007460C460AB101333360236863
:1025E000990642BF336802333360256815F006054B
:1025F00006D104F1190AE36832689B1AAB4226DC63
:1026000094F84320131E226818BF012392062BD48E
:1026100004F1430249463846C04701301ED02368C2
:10262000E568326803F00603042B08BFAD1AA368FF
:1026300022690CBF25EAE57500259342C4BF9B1AA9
:10264000ED1800261A34B5421AD1002008E0012303
:10265000524649463846C047013003D14FF0FF305B
:10266000BDE8F0870135C6E7E1185A1C302081F833
:102670004300224494F8451082F843100233C7E720
:102680000123224649463846C0470130E6D001368C
:10269000D9E700002DE9FF470C469146277E0C99AB
:1026A000782F80469A4604F1430207D8622F0AD851
:1026B000002F00F0D880582F00F0A38004F14206CC
:1026C00084F842703AE0A7F16303152BF6D801A015
:1026D00050F823F02D27000041270000BD26000000
:1026E000BD260000BD260000BD26000041270000D9
:1026F000BD260000BD260000BD260000BD2600004E
:102700004D280000712700002F280000BD26000082
:10271000BD2600006F280000BD26000071270000C4
:10272000BD260000BD260000372800000B681A1DDA
:102730001B680A6004F1420684F842300123A3E0DA
:10274000256808682E0600F104030AD505680B60A9
:10275000002D03DA2D236D4284F843305E480A23AE
:1027600019E015F0400F05680B6018BF2DB2EFE7B8
:102770000B682568181D0860280601D51D6802E051
:102780006906FBD51D8854486F2F0CBF08230A2308
:10279000002184F843106668A660002EA2BF21685D
:1027A00021F0040121600DB9002E4DD01646B5FB75
:1027B000F3F103FB1157C75D06F8017D2F46BB42BD
:1027C0000D46F4D9082B0BD12368DF0708D5236900
:1027D00061689942DEBF302306F8013C06F1FF36FE
:1027E000921B2261CDF800A04B4603AA2146404629
:1027F000FFF7E2FE01304CD14FF0FF3004B0BDE8EE
:10280000F087354884F8457023680E681F0656F82F
:10281000045B0E6014D5D90744BF43F02003236046
:102820001DB9236823F0200323601023B0E7236839
:1028300043F0200323607823284884F84530E3E7F9
:102840005E0648BFADB2E6E71646BBE70B682668F2
:1028500060691D1D0D6035061B6801D5186002E01A
:102860007106FBD51880002323611646BAE70B6872
:102870001A1D0A601E6862680021304600F040F8A8
:1028800008B1801B606063682361002384F84330D3
:10289000A8E72369324649464046D0470130ABD0CD
:1028A00023689B0713D4E068039B9842B8BF18467F
:1028B000A4E70123324649464046D04701309BD029
:1028C0000135E36803995B1AAB42F2DCEBE70025C4
:1028D00004F11906F5E700BF7D3100008E310000DC
:1028E00038B5064D0023044608462B60FDF776FDFB
:1028F000431C02D12B6803B1236038BD680300205C
:1029000001F0FF01102A2BDB10F0070F08D010F8A0
:10291000013B013A8B422DD010F0070F42B3F6D1A4
:10292000F0B441EA012141EA014122F007047FF0BD
:1029300000070023F0E80256083C85EA010586EA14
:10294000010685FA47F5A3FA87F586FA47F6A5FA50
:1029500087F68EB9EED1F0BC01F0FF0102F007025C
:1029600032B110F8013B013A83EA010313B1F8D107
:102970000020704701387047002D06BF35460338E8
:10298000073815F0010F07D1013015F4807F02BF21
:10299000013015F4C03F0130F0BC0138704700BF72
:1029A000884210B501EB020402D98442234607D8BD
:1029B000431EA14208D011F8012B03F8012FF8E7BC
:1029C000024401468A4200D110BD13F8014D02F8BD
:1029D000014DF7E70148FFF737BC00BF6003002057
:1029E0000148FFF732BC00BF6003002038B5054640
:1029F000002945D051F8043C0C1F002BB8BFE41847
:102A0000FFF7E8FF1F4A1368104633B9636014608C
:102A10002846BDE83840FFF7E3BFA3420BD9216841
:102A20006218934204BF1A685B68636004BF52185F
:102A300022600460ECE71A465B680BB1A342FAD946
:102A400011685018A0420BD12068014450188342ED
:102A50001160DDD118685B68536001441160D7E7ED
:102A600002D90C232B60D3E7206821188B4204BFC6
:102A700019685B68636004BF091821605460C7E788
:102A800038BD00BF54030020F8B5074614460E4673
:102A900021B9BDE8F8401146FFF7D8BB22B9FFF7CE
:102AA000A5FF25462846F8BD00F014F8A0420FD235
:102AB00021463846FFF7CAFB05460028F2D03146CA
:102AC0002246FFF783FB31463846FFF78FFFE9E7E1
:102AD0003546E7E751F8043C181F002BBCBF0B58E4
:102AE000C01870472E2E2F68616C2F7372632F6889
:102AF000616C5F696F2E63002E2E2F68616C2F73DF
:102B000072632F68616C5F63616C656E6461722EC5
:102B100063002E2E2F73645F6D6D632F73645F6D82
:102B20006D632E63003E3E3E005374617274205309
:102B300044206361726420696E7374616C6C0A0D69
:102B40000025733A20434D443535204661696C0AAF
:102B50000D0025733A2041434D44343120466169CC
:102B60006C0A0D0025733A2041434D443431205402
:102B7000696D656F7574206F6E20627573792C2096
:102B800072657370333220307825303878200A0D22
:102B90000025733A20434D443538204661696C0A5C
:102BA0000D005374617274204D4D4320496E73744F
:102BB000616C6C0A0D0025733A20434D443120535B
:102BC0005049204661696C202D204275737920722E
:102BD000657472792025640A0D0025733A20434DEF
:102BE00044312054696D656F7574206F6E20627575
:102BF00073790A0D0053442F4D4D43206361726475
:102C00002072656164790A0D0000000073645F73CF
:102C100070695F6F705F636F6E64006D6D635F738B
:102C200070695F6F705F636F6E640000000000008A
:102C30000A0000000C0000000D0000000F00000062
:102C4000140000001A0000001E0000002300000015
:102C5000280000002D0000003400000037000000B4
:102C60003C00000046000000500000000A00000088
:102C700064000000E80300001027000000000000CE
:102C80000000000000000000000000000A0000003A
:102C90000C0000000D0000000F00000014000000F8
:102CA000190000001E0000002300000028000000A2
:102CB0002D00000032000000370000003C00000042
:102CC00046000000500000002E2E2F73645F6D6DD3
:102CD000632F73645F6D6D635F7370692E6300258E
:102CE000733A205265616420626C6F636B73207469
:102CF000696D656F75740A0D0025733A2043524360
:102D00002064617461206572726F7220746F6B65EC
:102D10006E0A0D0025733A204F7574206F6620727D
:102D2000616E67652064617461206572726F7220E4
:102D3000746F6B656E0A0D0025733A20496E7661DB
:102D40006C6964204461746120526573706F6E73A6
:102D50006520546F6B656E20307825780A0D00254C
:102D6000733A20577269746520626C6F636B732CC1
:102D70002053445F4D4D435F5350495F4552525F6E
:102D80004352432C207265737020307825780A0DE9
:102D90000025733A20577269746520626C6F636B0B
:102DA000732053445F4D4D435F5350495F4552522A
:102DB0005F57522C207265737020307825780A0D89
:102DC0000025733A2053746F702077726974652000
:102DD000626C6F636B732074696D656F75740A0D37
:102DE000004E6F20534420436172642072657370FB
:102DF0006F6E7365207761732070726573656E7492
:102E00002E2E2E0025733A20636D64202530326407
:102E10002C206172672030782530386C582C205275
:102E2000312074696D656F75740D0A0025733A2041
:102E3000636D6420253032642C2061726720307805
:102E40002530386C782C207231203078253032785B
:102E50002C2052315F5350495F434F4D5F435243E3
:102E60000A0D0025733A20636D6420253032642CEE
:102E7000206172672030782530386C782C207231D0
:102E800020307825782C20523120494C4C45474140
:102E90004C5F434F4D4D414E440A0D0025733A207F
:102EA000636D6420253032642C2061726720307895
:102EB0002530386C782C20723120307825782C2001
:102EC0005231206572726F720A0D0025733A2063C9
:102ED0006D6420253032642C2061726720307825A3
:102EE00030386C782C2042757379207369676E6175
:102EF0006C20616C7761797320686967680A0D00DE
:102F000025733A20577269746520626C6F636B7326
:102F10002074696D656F75740A0D003C3C3C00734C
:102F200070695F6D5F73796E635F73746172745FF4
:102F3000726561645F626C6F636B007370695F6D73
:102F40005F73796E635F73746F705F7772697465B6
:102F50005F626C6F636B007370695F6D5F73796E36
:102F6000635F73746F705F6D756C74697772697489
:102F7000655F626C6F636B007370695F6D5F73791F
:102F80006E635F616474635F737461727400737005
:102F9000695F6D5F73796E635F73746172745F777D
:102FA000726974655F626C6F636B73007370695FE5
:102FB0006D5F73796E635F776169745F656E645F7F
:102FC0006F665F77726974655F626C6F636B7300C5
:102FD0007370695F6D5F73796E635F777269746533
:102FE0005F776F7264002E2E2F68616C2F7372638F
:102FF0002F68616C5F7370695F6D5F73796E632EAC
:1030000063002E2E2F68616C2F7372632F68616CC2
:103010005F6D63695F73796E632E63002E2E2F6878
:10302000706C2F736468632F68706C5F736468637F
:103030002E63002E2E2F68616C2F7372632F6861D0
:103040006C5F75736172745F73796E632E63004891
:10305000656C6C6F20776F726C640A002E2E2F687F
:10306000706C2F7274632F68706C5F7274632E6360
:10307000002E2E2F68706C2F736572636F6D2F6832
:10308000706C5F736572636F6D2E6300003000407B
:103090000034004000200141004001410000004395
:1030A0000004004300080043000C0043000000003F
:1030B0000000000000000000000000000000000010
:1030C000000000000C0030000000020000000000C2
:1030D000FE00FF0104446562756720496E697469EA
:1030E000616C697A65640A00417373657274204685
:1030F00061696C757265206174206C696E6520254C
:10310000642C2025733A2025730A0000000000007B
:1031100000000000000000000000000000000000AF
:10312000000000000000000000000000000000009F
:10313000000000000000000000000000000000008F
:10314000000000000000000000000000000000007F
:10315000000000000000000000000000000000006F
:10316000000000000000000000000000232D302BB4
:103170002000686C4C006566674546470030313278
:1031800033343536373839414243444546003031CF
:10319000323334353637383961626364656600002E
:1031A000F8B500BFF8BC08BC9E4670478902000015
:1031B000F8B500BFF8BC08BC9E4670476502000029
:1031C000FFFF0100FFFF00000C00002000000000D6
:1031D0002C3100004C3100000C31000000000000D8
:1031E00000000000000000000000000000000000DF
:1031F00000000000000000000000000000000000CF
:1032000000000000000000000000000000000000BE
:1032100000000000000000000000000000000000AE
:0C322000000000000000000000000000A2
:00000001FF
